:020000040000FA
:0400000025EF00F0F8
:0200080037D0EF
:0800180085D0046A036EFF0E9F
:100020000326042200D0D8A01200030E026EE70EB1
:1000300002D8F5D7026AFE0F016EE86A025AD8A00C
:1000400012000000010600D0F8D7F86A4F0EAF6E1C
:10005000240EAC6E900EAB6E0001070EB46E0F0E48
:10006000C16EC69AC00E926EE00E936EC00E946E74
:10007000956AE80E966E1FD19EAA1BD0060EAB1491
:1000800012E1E1CF29F0E2CF2AF02B2A1EEE80F018
:100090002B50E126000EE222AECFE7FF29C0E1FFA0
:1000A0002AC0E2FF1100AE50AE50AB98AB881100F1
:1000B0000AD0F2A408D0F294074A082A817A066A84
:1000C000D6CF05F0110011002B502C5C14E02C2A27
:1000D000E9CF01F0EACF02F00EEE80F02C50E926D5
:1000E000000EEA22EF50016E01C0E9FF02C0EAFFF4
:1000F000D880120004D0E868016ED8A01200120067
:100100002B6A2C6A9D8A9F8AF28EF28C12009D9A2D
:100110000EEE80F0000EEE6AE82EFDD72B6A2C6AF8
:100120009D8A1200F29ED8CF58FEE8CF59FEE0CF4C
:100130005AFEE9CF5BFEEACF5CFEE1CF5DFEE2CF87
:100140005EFED9CF5FFEDACF60FEF6CF61FEF7CF5D
:1001500062FEF5CF63FEF3CF64FEF4CF65FEA6CF5B
:1001600066FE01C067FE03C068FEF28E0001A19228
:100170001BA24AD025C0B2FF26C0B3FF0B4A0C2AEF
:100180000BA241D00B6A0C6A2750016E15083BE3A5
:10019000FA6AD8900136FA360136FA36AE0E0126E2
:1001A000010EFA22FB6A000EFB220150F96E32EFBB
:1001B00001F008EF01F00AEF01F00CEF01F00EEF93
:1001C00001F010EF01F012EF01F014EF01F016EF63
:1001D00001F018EF01F01AEF01F01CEF01F01EEF33
:1001E00001F020EF01F022EF01F024EF01F026EF03
:1001F00001F028EF01F02AEF01F02CEF01F02EEFD3
:1002000001F030EF01F02ED00B6A0C6A2BD02AD00F
:10021000807428D0807226D0807024D0807622D03E
:10022000807820D0807A1ED084701CD084721AD03E
:10023000847418D0817816D0817614D0817412D04D
:10024000817210D081700ED0837E0CD0837C0AD056
:10025000837A08D0837806D0827A04D0827802D05C
:10026000837600D0F29E58CED8FF59CEE8FF5ACE02
:10027000E0FF5BCEE9FF5CCEEAFF5DCEE1FF5ECE44
:10028000E2FF5FCED9FF60CEDAFF61CEF6FF62CE2D
:10029000F7FF63CEF5FF64CEF3FF65CEF4FF66CEC5
:1002A000A6FF67CE01F068CE03F0F28E10009EA884
:1002B000FED7AD6E1200939A8A8A0A0EAEDE939A2A
:1002C0008A9AF7D996EC03F01C6A780E226E22C047
:1002D00024F0236AD8902436286A12DF18DFCD6A0A
:1002E000F294F28A870ED56EB16AA192A082B26AA8
:1002F000B36AD08EA292B10EB16EE6DE0D6EB60E6E
:100300000D5C07E3FE0E0D5C02E30DD102D00F6A17
:100310000AD10DAE20D00F6A850E0D5C05E10DC02F
:100320000FF01068116816D0950E0D5C05E10DC038
:100330000FF0126813680ED0B50E0D5C05E10DC00C
:100340000FF01468156806D0D50E0D5C03E10DC0E2
:100350000FF01668E8D00F5202E1E5D0E4D0850E28
:100360000F5C3BE1102803E10DC010F035D00DC04B
:1003700011F02B0E105C18E36B0E105C15E21B8065
:10038000B190216A1B92D6CF05F0D7CF06F023504B
:100390000524176E24500620186E000E0720196ED3
:1003A000000E08201A6E17D07C0E105C05E10101CA
:1003B000AD918C9000010FD07D0E105C05E1010124
:1003C000AD938C92000107D07E0E105C03E1010119
:1003D000AD958C9400011068A6D0950E0F5CD8A442
:1003E0008ED0122803E10DC012F088D00DC013F09A
:1003F000135233E12B0E125C18E36B0E125C15E204
:100400001B80B1901B92216AD6CF05F0D7CF06F0A2
:1004100023500524176E24500620186E000E072066
:10042000196E000E08201A6E17D07C0E125C05E1C2
:100430000101AD918C9000010FD07D0E125C05E1A1
:100440000101AD938C92000107D07E0E125C03E196
:100450000101AD958C94000151D02B0E125C36E356
:100460006B0E125C33E22B0E125C206E1B9000EEC2
:100470002DF02050EB50806E00EE6DF02050EB50D0
:100480000E6E0E8A81AA0E9A0EC081FF00EEADF0AC
:100490002050EB50826E00EEEDF02050EB50006EDD
:1004A0000101AD510024836E01EE2DF02050EB5080
:1004B000846E12C021F02852000107E001EE6DF0B9
:1004C0002050EB50276E1B82B18017D07C0E125C3F
:1004D00005E10101AD818C8000010FD07D0E125C21
:1004E00005E10101AD838C82000107D07E0E125C14
:1004F00003E10101AD858C840001126814D0B50EB2
:100500000F5C09E1142803E10DC014F003D00DC005
:1005100015F035D808D0D50E0F5C05E1162803E19B
:100520000DC016F016D81BA013D0D6CF05F0D7CF2C
:1005300006F01750055C18500658195007581A5005
:10054000085808501A18D8B0800A02E7D9D81B906A
:10055000D4D616520EE0B19016C028F028C026F06E
:10056000256AD890263625C0B2FF26C0B3FFB180D9
:1005700004D0286A256A266AB190166812001E0EF9
:10058000145C0CE115C022F0225202E11B9005D050
:1005900022C024F0236AD890243689D01F0E145C20
:1005A00018E11550285C14E015520EE0B19015C00A
:1005B00028F028C026F0256AD890263625C0B2FF3C
:1005C00026C0B3FFB18004D0B190286A256A266A9C
:1005D0006ED0420E145C07E1155203E11C9069D8FD
:1005E00001D01C8064D0640E145C1DE115B08084C1
:1005F00015A0809415B2808215A2809215B48080D7
:1006000015A4809015B6808615A6809615B88088AA
:1006100015A8809815BA808A15AA809A15BC84807E
:1006200015AC849044D0650E145C1DE115B0848235
:1006300015A0849215B2848415A2849415B481887F
:1006400015A4819815B6818615A6819615B8818462
:1006500015A8819415BA818215AA819215BC818052
:1006600015AC819024D0660E145C1DE115B0838E0C
:1006700015A0839E15B2838C15A2839C15B4838A22
:1006800015A4839A15B6838815A6839815B8828A0F
:1006900015A8829A15BA828815AA829815BC8386F5
:1006A00015AC839604D07B0E145CD8B402D81468C1
:1006B00012001B6A076A086A899489928990899650
:1006C0008998899A8D908D928D948A988A968A9429
:1006D0008A928A908C9E8C9C8C9A8C988B9A8B9800
:1006E0008C968C908C928C940101AD6B780E226E5E
:1006F00022C024F0236AD8902436286A0001120010
:1007000089948992899089968998899A8D908D92F9
:100710008D948A988A968A948A928A908C9E8C9CD0
:100720008C9A8C988B9A8B988C961200150E2D6E45
:100730000A0E6D6EAD6BE00EED6F070E01012D6FB1
:10074000110E2E6E0A0E6E6E0001AE6BE00EEE6F95
:10075000070E01012E6F130E2F6E0A0E6F6E000131
:10076000AF6BE00EEF6F070E01012F6F080E306EBA
:100770000A0E706E0001B06BE00EF06F070E010103
:10078000306F180E316E0A0E716E0001B16BE00E03
:10079000F16F070E0101316F326A0A0E726E0001AD
:1007A000B26BE00EF26F070E0101326F380E336E3E
:1007B0000A0E736E0001B36BE00EF36F070E0101BA
:1007C000336F346A0A0E746E0001B46BE00EF46F7E
:1007D000040E0101346F356A0A0E756E0001B56BA7
:1007E000E00EF56F0101356B366A1A0E766E000168
:1007F000B66BE00EF66F0101366B376A020E776E4C
:100800000001B76BE00EF76F0101376B386A060E17
:10081000786E0001B86BE00EF86F0101386B396A31
:10082000020E796E0001B96BE00EF96F0101396BB0
:100830003A6A030E7A6E0001BA6BE00EFA6F01019C
:100840003A6B3B6A7B6A0001BB6B200EFB6F0101B8
:100850003B6B3C6A7C6A0001BC6BFC6B01013C6B2E
:100860003D6A7D6A0001BD6B100EFD6F01013D6B9D
:100870003E6A7E6A200E0001BE6FFE6B01013E6B78
:100880003F6A7F6A100E0001BF6FFF6B01013F6B73
:10089000150E406E0A0E0001806FC06BE00E010164
:1008A000006F070E406F110E416E0A0E0001816F3E
:1008B000C16BE00E0101016F070E416F130E426E16
:1008C0000A0E0001826FC26BE00E0101026F070E7B
:1008D000426F100E436E0A0E0001836FC36BE00E71
:1008E0000101036F070E436F180E446E0A0E0001DC
:1008F000846FC46BE00E0101046F070E446F456AFC
:100900000A0E0001856FC56BE00E0101056F070E31
:10091000456F380E466E0A0E0001866FC66BE00EFC
:100920000101066F070E466F476A0A0E0001876FC6
:10093000C76BE00E0101076F040E476F486A0A0E8D
:100940000001886FC86BE00E0101086F486B496AAF
:100950001A0E0001896FC96BE00E0101096F496B26
:100960004A6A020E00018A6FCA6BE00E01010A6F2B
:100970004A6B4B6A080E00018B6FCB6BE00E0101D6
:100980000B6F4B6B4C6A030E00018C6FCC6BE00E4F
:1009900001010C6F4C6B4D6A020E00018D6FCD6B27
:1009A000200E01010D6F4D6B4E6A00018E6BCE6BF8
:1009B00001010E6F4E6B4F6A0A0E00018F6FCF6BF5
:1009C000200E01010F6F4F6B506A0A0E0001906FED
:1009D000D06B200E0101106F010E506F516A0A0E8C
:1009E0000001916FD16B200E0101116F516B526AA2
:1009F000080E0001926FD26BE00E0101126F526B74
:100A0000536A020E0001936FD36B200E0101136F26
:100A1000536B546A060E0001946FD46B200E0101D3
:100A2000146F546B100E556E080E0001956FD56B48
:100A3000E00E0101156F010E556F180E566E0A0E6D
:100A40000001966FD66BA00E0101166F050E566F52
:100A5000120E576E0A0E0001976FD76B200E010120
:100A6000176F050E576F020E586E0001986FD86B06
:100A7000E00E0101186F050E586F220E596E00012D
:100A8000996BD96BE00E0101196F050E596F180EA5
:100A90005A6E080E00019A6FDA6BE00E01011A6FB0
:100AA000050E5A6F020E5B6E00019B6FDB6B200E12
:100AB00001011B6F050E5B6F100E5C6E020E0001D4
:100AC0009C6FDC6B280E01011C6F050E5C6F150E10
:100AD0005D6E0A0E00019D6FDD6BE80E01011D6F5A
:100AE000070E5D6F110E5E6E0A0E00019E6FDE6BCB
:100AF000E80E01011E6F070E5E6F130E5F6E0A0E89
:100B000000019F6FDF6BE80E01011F6F070E5F6F23
:100B1000100E606E0A0E0001A06FE06BE80E01017E
:100B2000206F070E606F300E616E0A0E0001A16F1C
:100B3000E16BE80E0101216F070E616F626A0A0E18
:100B40000001A26FE26BE80E0101226F070E626FD7
:100B5000380E636E0A0E0001A36FE36BE80E01010D
:100B6000236F070E636F646A0A0E0001A46FE46BC3
:100B7000E80E0101246F040E646F656A0A0E00011D
:100B8000A56FE56BE80E0101256F656B666A1A0EAD
:100B90000001A66FE66BE80E0101266F666B676ABF
:100BA000020E0001A76FE76BE80E0101276F676B6C
:100BB000686A060E0001A86FE86BE80E0101286F55
:100BC000686B696A020E0001A96FE96BE80E01010A
:100BD000296F696B6A6A030E0001AA6FEA6BE80E5F
:100BE00001012A6F6A6B6B6A0001AB6BEB6B280E1D
:100BF00001012B6F6B6B6C6A0001AC6BEC6B080E28
:100C000001012C6F6C6B150E6D6F130E6E6F120E53
:100C10006F6F130E706F140E716F030E726F0E0EE6
:100C2000736F130E746F120E756F0E0E766F090EC2
:100C3000776F0B0E786F0E0E796F150E7A6F0B0EA5
:100C40007B6F140E7C6F150E7D6F7E6F080E7F6FAD
:100C5000150E806F010E816F120E826F010E836F71
:100C6000030E846F010E856F030E866F876F040E6F
:100C7000886F010E896F020E8A6F030E8B6F040E50
:100C80008C6F060E8D6F010E8E6F080E8F6F010E2A
:100C9000906F916F926F050E936F946F080E956F22
:100CA000090E966F010E976F986F060E996F070EDB
:100CB0009A6F080E9B6F010E9C6F9D6F9E6F050EC5
:100CC0009F6FA06F080EA16F0C0EA26F010EA36F95
:100CD0000A0EA46F080EA56FA66F110EA76FA86F5E
:0E0CE000A96FAA6FAB6FAC6F00011200FFD7B7
:020000040030CA
:0300010006160ED2
:020005008580F4
:060008000FC00FE00F40E5
:00000001FF
